:0200000270008C
:10800000807F0020398507006185070063850700B0
:108010006585070067850700698507000000000087
:108020000000000000000000000000006B85070059
:108030006D850700000000006F850700718507004F
:108040007385070073850700738507007385070034
:108050007385070073850700738507007385070024
:108060007385070073850700738507007385070014
:108070007385070081C307007385070073850700B8
:108080007385070099C7070073850700738507008C
:1080900041C40700738507002DC1070073850700E1
:1080A00073850700738507007385070073850700D4
:1080B00073850700738507000000000000000000C2
:1080C00073850700738507007385070073850700B4
:1080D00073850700738507007385070000000000A3
:1080E0000000000000000000000000000000000090
:1080F0000000000000000000000000000000000080
:10810000000000000000000000000000000000006F
:10811000000000000000000000000000000000005F
:1084000010B5054C237833B9044B13B10448AFF3CE
:1084100000800123237010BD882C00200000000084
:1084200090CF070008B5034B1BB103490348AFF3D6
:10843000008008BD000000008C2C002090CF0700B9
:10844000154B002B08BF134B9D46A3F5803A002126
:108450008B460F461348144A121A00F063F80F4B6C
:10846000002B00D098470E4B002B00D098470020DF
:10847000002104000D000D48002802D00C48AFF385
:10848000008000F02BF82000290004F0E5F900F04E
:1084900011F800BF00000800807F002000000000ED
:1084A00000000000882C0020B438002000000000EC
:1084B0000000000008B5074B044613B10021AFF3DC
:1084C0000080054B1868836A03B19847204600F086
:1084D00031F800BF0000000024CC070070B50D4D3E
:1084E0000D4C641BA4100026A64209D10B4D0C4C68
:1084F00004F08CFB641BA4100026A64205D170BDBD
:1085000055F8043B98470136EEE755F8043B984789
:108510000136F2E7682C0020682C0020682C00202F
:108520006C2C002002440346934200D1704703F8AC
:10853000011BF9E7FEE700BF0649074A074B9B1AF4
:1085400003DD043BC858D050FBDC03F003FEFFF70B
:1085500077FF00009CCF0700002C0020882C002013
:10856000FEE7FEE7FEE7FEE7FEE7FEE7FEE7FEE7E3
:10857000FEE7FEE770B5EFF3108672B60D4A946819
:108580000123A4B993600C4B0C4DD3F88010294003
:108590001160C3F88050D3F8841051604FF0FF325F
:1085A000C3F88420047006B962B6002070BD037061
:1085B000F9E700BF7434002000E100E0FC06FFBCD6
:1085C0002DE9F04FC9B008AA01F1400514464B78D7
:1085D0000E781B0443EA0663CE7833438E78043169
:1085E00043EA06238D4244F8043BF0D11024916BFA
:1085F00016464FEAF14383EA714383EA9123716A95
:10860000366852F8045F31440B444FEAB54181EAC1
:10861000F51181EAD50101340B44402CD363E6D136
:10862000D0E914E30093836D0193C36D0293036E4D
:108630000393436E0493836E0593C36E0693DDE943
:10864000057BDDE9031CDDE901592B4B009E0793F7
:1086500074464FF00008079B53F8042B07934FEA2A
:10866000F12383EAB11383EA716A08AB53F8283027
:108670001A440AEB020327EA010A01EA0C028AEA19
:1086800002021A444FEA743A86EA05035A448AEA17
:10869000B40A06EA050B234083EA0B038AEAB45ABC
:1086A00008F101089A44B8F1400F02EB0903BB46F8
:1086B0005244A94619D172440265009A2244426587
:1086C000019A32448265029A2A44C265039A1A4486
:1086D000049B02660B444366059B63448366069BCA
:1086E0003B44C36649B0BDE8F08F674635468C46CB
:1086F000264619461446AEE750CE07002DE9F04F46
:1087000093B0CDE9002002A892F90020B1E8005E04
:1087100006B4AAFB09124FF00003EBFB69234FF0EC
:108720000004ECFB69344FF00005EEFB69454FF0A7
:108730000006EBFB6A63ECFB6A3449185241764150
:108740005B41A9FB09784FF0000949F1000918EBDA
:108750000108A0E88001AAFB0A78574158EB0608F7
:10876000A0E88001EEFB6A454FF0000A4AF1000ADA
:108770004FF00001ECFB6B14EEFB6B454FF0000279
:10878000EEFB6C255FEA59094941644152416D4154
:1087900049F10009EBFB6B3A1AEB010AA0E8080467
:1087A000ACFB0C6A66415AEB020AA0E84004AEFB3F
:1087B0000E6A6E415AEB090AA0E8400406BC052A7D
:1087C00000F0E680A0F11400A1F11401B1E8E0434B
:1087D000A5FB0E344FF00005E6FB6E454FF000069A
:1087E000E7FB6E564FF00007E8FB6E674FF000089E
:1087F000E9FB6E784FF00009DB1864416D4176416A
:108800007F4158EB080859F1000950F804CB13EBED
:108810000C0350F804CB54EB0C0450F804CB55EB8C
:108820000C0550F804CB56EB0C0650F804CB57EB74
:108830000C0758F1000859F10009A0F11400EEFBF3
:108840000E89A0E8F803062A00F0A280A0F1180023
:10885000A1F11801B1E8E047A5FB0E344FF0000587
:10886000E6FB6E454FF00006E7FB6E564FF0000743
:10887000E8FB6E674FF00008E9FB6E784FF00009E7
:10888000EAFB6E894FF0000ADB1864416D417641C6
:108890007F4158EB080859EB09095AF1000A50F8D2
:1088A00004CB13EB0C0350F804CB54EB0C0450F83E
:1088B00004CB55EB0C0550F804CB56EB0C0650F8E6
:1088C00004CB57EB0C0750F804CB58EB0C0859F1CC
:1088D00000095AF1000AA0F11800EEFB0E9AA0E878
:1088E000F807072A54D0A0F11C00A1F11C01B1E83F
:1088F000E04FA5FB0E344FF00005E6FB6E454FF050
:108900000006E7FB6E564FF00007E8FB6E674FF07E
:108910000008E9FB6E784FF00009EAFB6E894FF022
:10892000000AEBFB6E9A4FF0000BDB1864416D41BF
:1089300076417F4158EB080859EB09095AEB0A0ABE
:108940005BF1000B50F804CB13EB0C0350F804CB95
:1089500054EB0C0450F804CB55EB0C0550F804CB49
:1089600056EB0C0650F804CB57EB0C0750F804CB31
:1089700058EB0C0850F804CB59EB0C095AF1000ADB
:108980005BF1000BA0F11C00EEFB0EABA0E8F80FB2
:10899000009B0198D3F8AC3002A9984713B0BDE80A
:1089A000F08F00EB81010023884200D3704751F81B
:1089B000042D43EA52030B60D307F5E710B5013AE3
:1089C00052B2130601D5002010BD50F8224051F8D4
:1089D00022309C4205D802F1FF32F2D24FF0FF3034
:1089E000F2E70120F0E710B500235CB2A24200DC00
:1089F00010BD51F8234040F823400133F5E7013919
:108A000010B549B2041D0A06CBB204D4013954F89A
:108A10002120002AF7D001335BB273B103F1804209
:108A2000013A50F82220002022B9013B00EB431309
:108A300018B210BD52080130F6E71846F9E74A119E
:108A4000012350F8220001F01F0103FA01F1084050
:108A5000704710B500231A465CB2A14203DCB2FA9B
:108A600082F0400910BD50F8234001332243F3E760
:108A7000002310B51C465AB2914200DC10BD40F8EC
:108A800023400133F7E72DE9F04FA5B01D4604ABB5
:108A9000CDE902318146294610461746FFF7AFFF60
:108AA000C0EB851004B2002C2646B8BF04F11F06A7
:108AB000634246F3471603F01F0304F01F0814A88F
:108AC00058BFC3F100083146FFF7D2FFB8F1000FDD
:108AD00030B22DDD14AB002203EB8000C8F1200C76
:108AE00013469D4219D82FB27B00019314AB03EBC0
:108AF000870705F1FF3824AB012603EB8808002C1B
:108B000054DA24AB03EB86062A4656F8881C4846FE
:108B1000FFF769FF25B0BDE8F08F57F8236006FA2C
:108B200008F10A4340F8042B013326FA0CF2D8E787
:108B300014AB2A46394603EB8000FFF754FFD2E717
:108B40000FFA82FE5AF8883C53F82EB024AB03EBA0
:108B50008202013052F8403C0B44BBEB030334BFAC
:108B6000012200229B4518BF11465CF8882C42F870
:108B70002E30019B42B29A42E2DB731A5E422946D2
:108B800014A85E41FFF70DFF24AB03EB85032946D4
:108B900053F8402C58F8403C384643EAC273013C35
:108BA00048F8403C24B2FFF7FCFEA8E724AB0020C5
:108BB000C6F1010C014603EB860A03EB8C0CD8E7E7
:108BC0002DE9F04F08B4F8CA04B451F8042BA3FB04
:108BD000028940F8048B4FF0000AE4FB629A4FF0E0
:108BE000000BE5FB62AB4FF0000CE6FB62BC4FF004
:108BF000000EE7FB62CE51F8042B4FF00008E3FBB8
:108C0000628940F8048BE4FB629AE5FB62ABE6FB09
:108C100062BCE7FB62CE51F8042B4FF00008E3FB87
:108C2000628940F8048BE4FB629AE5FB62ABE6FBE9
:108C300062BCE7FB62CE51F8042B4FF00008E3FB67
:108C4000628940F8048BE4FB629AE5FB62ABE6FBC9
:108C500062BCE7FB62CE51F8042B4FF00008E3FB47
:108C6000628940F8048BE4FB629AE5FB62ABE6FBA9
:108C700062BCE7FB62CE40F8049B40F804AB40F8CE
:108C800004BB40F804CB40F804EB0CBC052B00F00F
:108C90001E810C68A0F11400A1F11401A2F11402CC
:108CA00052F804EB4FF0000550F8046BE4FB6E56ED
:108CB00052F804EB50F8047BE4FB6E6752F804EBC7
:108CC00050F8048BE4FB6E7852F804EB50F8049BE8
:108CD000E4FB6E8952F804EB50F804ABE4FB6E9AA7
:108CE000A0F1140052F8044B51F804EB4FF0000CC3
:108CF000E4FB6EC540F804CB51F804EBE4FB6E5680
:108D000040F8045B51F804EBE4FB6E6740F8046B39
:108D100051F804EBE4FB6E7840F8047B51F804EB67
:108D2000E4FB6E8940F8048B51F804EBE4FB6E9A87
:108D3000A0E80006062B00F0CA800C68A0F118001D
:108D4000A1F11801A2F1180252F804EB4FF000054E
:108D500050F8046BE4FB6E5652F804EB50F8047BB9
:108D6000E4FB6E6752F804EB50F8048BE4FB6E787A
:108D700052F804EB50F8049BE4FB6E8952F804EBC4
:108D800050F804ABE4FB6E9A52F804EB50F804BBC5
:108D9000E4FB6EABA0F1180052F8044B51F804EB61
:108DA0004FF0000CE4FB6EC540F804CB51F804EB27
:108DB000E4FB6E5640F8045B51F804EBE4FB6E678D
:108DC00040F8046B51F804EBE4FB6E7840F8047B48
:108DD00051F804EBE4FB6E8940F8048B51F804EB86
:108DE000E4FB6E9A40F8049B51F804EBE4FB6EAB95
:108DF000A0E8000C072B6AD008B40C68A0F11C0096
:108E0000A1F11C01A2F11C0252F804EB4FF0000585
:108E100050F8046BE4FB6E5652F804EB50F8047BF8
:108E2000E4FB6E6752F804EB50F8048BE4FB6E78B9
:108E300052F804EB50F8049BE4FB6E8952F804EB03
:108E400050F804ABE4FB6E9A52F804EB50F804BB04
:108E5000E4FB6EAB52F804EB50F804CBE4FB6EBCC1
:108E6000A0F11C0052F8044B51F804EB4FF0000342
:108E7000E4FB6E3540F8043B51F804EBE4FB6E561E
:108E800040F8045B51F804EBE4FB6E6740F8046BB8
:108E900051F804EBE4FB6E7840F8047B51F804EBE6
:108EA000E4FB6E8940F8048B51F804EBE4FB6E9A06
:108EB00040F8049B51F804EBE4FB6EAB40F804ABC4
:108EC00051F804EBE4FB6EBCA0E8001808BCBDE858
:108ED000F08F30B51C4691B0054693F900306846D6
:108EE000FFF76EFED4F8AC3069462846984711B0BB
:108EF00030BDF0B5154689B01C4607460E461A46E9
:108F000029466846FFF7FAFB23466A463946384643
:108F1000FFF7DFFF23462A4669466846FFF7D9FF79
:108F200023466A4631463046FFF7D3FF09B0F0BD0D
:108F3000C3F10803DB0070B50133002403A500BFB3
:108F40005B1920C940CAAD1B20C0184720C940CAC0
:108F5000B54120C020C940CAB54120C020C940CA7F
:108F6000B54120C020C940CAB54120C020C940CA6F
:108F7000B54120C020C940CAB54120C020C940CA5F
:108F8000B54120C06441B4FA84F0400970BD00BF0F
:108F9000C3F10803DB0070B50133002403A500BF53
:108FA0005B1920C940CAAD1920C0184720C940CA62
:108FB000754120C020C940CA754120C020C940CA9F
:108FC000754120C020C940CA754120C020C940CA8F
:108FD000754120C020C940CA754120C020C940CA7F
:108FE000754120C06441204670BD00BFF0B5082225
:108FF00089B00C460646FFF7F6FCCB6A03930B6B71
:1090000004934B6B05938B6B0693CB6B07930027F5
:1090100008236A4669466846CDE901770097FFF75D
:10902000B7FF082305466A4631463046FFF7B0FFD2
:10903000236B0393636B0493A36B0593E36B05446A
:10904000CDE906376A46082369466846FFF7A0FF60
:10905000082305446A4631463046FFF799FF236AE4
:109060000093636A0193A36A0293A36B0693E36B75
:109070000793054408236A4631463046CDE9047714
:109080000397FFF785FF636A0093A36AA26B0193BE
:10909000E36A02930492636BE26B0393CDE90523C9
:1090A000236A0793054408236A4631463046FFF792
:1090B0006FFFE36A0093236B0193636B0293236A50
:1090C0000693A36A0793054408236A46314630464F
:1090D000CDE904770397FFF72BFF236B0093636BB6
:1090E0000193A36B0293E36B0393636A0693E36AB2
:1090F00007932D1A08236A4631463046CDE9047796
:10910000FFF716FF636B0093A36B0193E36B02936E
:10911000236A0393636A0493A36ACDE90537236B3B
:1091200007932D1A08236A4631463046FFF700FFA1
:10913000A36B0093E36BCDE90137636A0393A36AE2
:109140000493E36ACDE90537636B07932D1A08236F
:109150006A4631463046FFF7EBFE2D1A0D4C0FD410
:1091600035B9082231462046FFF728FC01280FD0E8
:109170000823224631463046FFF7DAFE2D1AEFE784
:109180000823224631463046FFF702FF2D18F7D458
:1091900009B0F0BD68CC070070B5036813F0010595
:1091A0000646144605D013460A460146FFF7F0FE70
:1091B000054621463046FFF7F4FB45B104F18042F5
:1091C000013A56F8223043F0004346F8223070BD91
:1091D000F0B50F46A1B006461946384615461C465E
:1091E000FFF737FC20B13046FFF742FC21B0F0BD5D
:1091F000224639466846FFF7F6FB294608A8FFF7DE
:10920000F2FB10A82146FFF733FC012318A81093A6
:10921000FFF72EFC224608A96846FFF7CFFB28B9C6
:10922000224610A93046FFF7DEFBDFE7009BDA0796
:1092300009D421466846FFF7B4FB2246294610A808
:10924000FFF7AAFFE6E7089BDB0707D4214608A83B
:10925000FFF7A7FB2246294618A8F1E70028234676
:109260001CDD08AA69466846FFF762FE214668468B
:10927000FFF797FB224618A910A8FFF79FFB0028CD
:1092800005DA10A923462A460846FFF781FE10A9F1
:10929000234618AA0846FFF74BFECEE708A96A4600
:1092A0000846FFF745FE214608A8FFF77AFB22464D
:1092B00010A918A8FFF782FB002805DA18A9234691
:1092C0002A460846FFF764FE18A9234610AA084656
:1092D000FFF72EFEBEE770B59DF910401E462346EF
:1092E0000546FFF725FE38B1234632462946284673
:1092F000BDE87040FFF74CBE70BD2DE9F0438BB068
:109300001446129D15F9046B00961F468046894647
:109310002B460246214602A8FFF7DDFF02A9129A5A
:109320000846FFF7EBF9129B02AA41464046FFF7B9
:10933000D0FD129B02AA21462046FFF7CAFD2B460C
:109340004A46394638460096FFF7C5FF129A394615
:1093500002A8FFF7D3F902A92B4642460846009619
:10936000FFF7B9FF02A92B46224608460096FFF7F1
:10937000B2FF2B464246214620460096FFF7ABFF40
:10938000129B224649464846FFF7A3FD2B4602AAF8
:10939000414620460096FFF79EFF129B2246394623
:1093A0003846FFF796FD2B464A4639463846009622
:1093B000FFF791FF324602A92046FFF714FB0BB0DE
:1093C000BDE8F0832DE9F04FEBB09346749F059113
:1093D000B7F9022097F9004012F11F0148BF02F1CE
:1093E0003E0141F347120292013A4FEA82096AA90B
:1093F00012AE82460DF1280801EB0900002140F869
:10940000C01C46F8221048F8221097F90110304687
:109410000D460A46002A40F0268103EB4103002D49
:1094200040F0278121463046FFF713FB002840F02B
:1094300016814046FFF70DFB0490002840F00F8195
:1094400007F12403029A039331461846FFF7B6FA50
:10945000012840F00481029A03984146FFF7AEFAD2
:10946000012840F0FC8042AEDDE902323046FFF7D1
:10947000AFFE6AAB9944B7F9023049F8605C13F16A
:109480001F0548BF03F13E05DA1D48BF03F10E0278
:109490006D11D2100DF5A4784FFA85F99345494620
:1094A000404628BF9346FFF7E3FA059B08EB0B0203
:1094B0005B4405998B4240F0E280B7F902304FEAF5
:1094C000CB0B9B4515D9ABEB030B08EB85050022B5
:1094D000CBF12000A845C0F0D7804A46414603980A
:1094E000FFF76CFA012804D04B46039A4046FFF779
:1094F0001FFD5AAD2846029B324652A9FFF760FB7A
:10950000DDE90232294652A8FFF7BDFA2846029B40
:10951000324612A9FFF754FB4FEA840BDDE9023211
:1095200029464AA8FFF7AFFA05EB0B092246514638
:109530002846FFF758FA07F144080AEB0B014846A2
:10954000FFF751FA41462AA8FFF74DFA08EB0B0145
:1095500022A8FFF748FA3B1D29462AAA3046009464
:109560000593FFF7B8FE4B462A4622A92AA8009782
:10957000FFF7C3FE23463A1D31463046FFF728FE6B
:109580003246494628463B46FFF7B3FC0023029982
:1095900052A8CDE90638CDE908A5FFF730FA0299BF
:1095A00080464AA8FFF72BFA8045B8BF80461FFACD
:1095B00088F808F1FF352DB2294652A8FFF73FFA87
:1095C000294610F1000A4AA818BF4FF0010AFFF718
:1095D00036FA002814BF022300234AEA030A0DF1D9
:1095E0001809224659F82A500DF1E809294648463B
:1095F0000DF1C80AFFF7F7F905EB0B015046FFF72D
:10960000F2F921463046FFF733FA01234293A8F1DD
:1096100002080FFA88F8B8F1000F3EDA2346059ADF
:1096200031463046FFF7D4FD3B4632465146484668
:10963000FFF75FFC029A03984946FFF7BFF901283C
:1096400004D0DDE902324846FFF772FC013C64B207
:1096500012AA230663D5049BB3FA83F56D09284645
:109660006BB0BDE8F08F013A13F802C002F800C0F9
:10967000D0E6013D13F8012D08F80520CFE613F8D8
:10968000011D02F8011D14E755F8041D21FA0BF322
:1096900013432B6001FA00F21CE73B463246D7F831
:1096A000A45051464846A847414652A8FFF7C7F97B
:1096B0004146051C4AA818BF0125FFF7C0F900283C
:1096C00014BF022300231D4306AB53F825501DB3DE
:1096D000224629462AA8FFF786F905EB0B0122A8A6
:1096E000FFF781F93B46324622A92AA8FFF701FC81
:1096F000059B00942AAA49461AA8FFF7ECFD534699
:109700004A4622A92AA80097FFF7F7FD3B461AAA66
:1097100031463046FFF7DDFB08F1FF3879E752F8B4
:10972000241059F824304B40049919430491013C0A
:109730008FE770B59DF910401E4623460546FFF79A
:1097400027FC30B9224629463046FFF737F9012871
:1097500007D02346324629462846BDE87040FFF729
:10976000E7BB70BD2DE9F04115468AB00446884636
:109770001C22002103A8FEF7D5FE2E1D95F90070CE
:1097800003232A46414620460293FEF7B7FF33469D
:1097900002AA214620460097FFF79DFD2B46424630
:1097A00021462046FFF795FB0097334605F18402DA
:1097B00021462046FFF7BDFF0AB0BDE8F0812DE944
:1097C000F04793F9006092B004468946104631464E
:1097D00015469846FFF73DF9002840F09180424633
:1097E00049460AA8FEF78AFF43460AAA214602A86C
:1097F000FFF76FFB0AA908464246FEF77FFF434684
:109800002A4649464846FFF764FB08F104074246EA
:1098100029462846FEF772FF3B462A462146204647
:109820000096FFF786FF3B462A46294628460096C3
:10983000FFF77FFF3B462A46214628460096FFF762
:109840004AFD43462A4621462046FFF742FB3B4657
:109850002246214628460096FFF76BFF3B460096BE
:109860002A4621462046FFF764FF2368DB074AD5D6
:1098700033463A4621462046FFF78AFB3146824668
:109880002046FFF78EF806F18043013B54F8230091
:1098900040EACA7044F82300424621462846FEF7B3
:1098A0002DFF3B4602AA294628460096FFF713FDE6
:1098B0003B4602AA294628460096FFF70CFD02A95E
:1098C00008463B462A460096FFF705FD434602AA96
:1098D00021462046FFF7FDFA0AAA3B4610462146DC
:1098E0000096FFF7F8FC324629462046FFF77BF842
:1098F00049462846FFF777F80AA94846FFF773F864
:1099000012B0BDE8F08731462046FFF74AF8C3E7BA
:1099100010B5012203680446984710B1A368013BC3
:10992000A36010BD10B50B689A684B680024C0E9AD
:109930000243C0E9002294782344036192F9034072
:10994000234443614B68036101F10C034361537885
:1099500003F0C003802B04BF0431016110BD4368D4
:109960001A44426011B101399A4201D10120704775
:1099700013F8010B01F8010FF6E72DE9F347002575
:1099800080460F462E462C46D8F8083023B30DF1FA
:1099900007014046FFF7BCFFF0B19DF807C00CF08F
:1099A0007F025FFA82F9A4F12003C4F1200109FAD1
:1099B00003F329FA01F109FA04F20B431CF0800FBA
:1099C00045EA020546EA030604F1070402D1C7E9A5
:1099D000005602E0462CD7D1002002B0BDE8F08747
:1099E000F7B50F4669461646FFF7C7FFB0B1DDE988
:1099F0000013002501F001044A0842EAC37254EA48
:109A000005014FEA530314BFDD431D463B7914BFE4
:109A1000D4431446082B03D1C6E9004503B0F0BD7A
:109A2000042B08D134602246D317AB4206BFA242B2
:109A300001200020F2E7022B03D123B233801AB2B7
:109A4000F2E7012B03D163B233705AB2ECE7002086
:109A5000E4E773B50C4669461646FFF78EFF68B11A
:109A60002379082B0CD1DDE90045C6E90045DDE985
:109A70000023AB4206BFA2420120002002B070BD0D
:109A8000042B04D1009B33601C460025EFE7022B1A
:109A90004FF0000004D1009B33809CB20546E6E7FE
:109AA000012BEBD1009B337003F0FF04F6E737B5D1
:109AB0000D4669461446FFF760FF30B12A79082A3F
:109AC000DDE9003103D1C4E9003103B030BD042A1F
:109AD00018464FEAE37108D123601A460B468B42C1
:109AE00006BF824201200020EFE7022A04D11BB208
:109AF00023801AB2D317F2E7012A03D15BB2237095
:109B00005AB2F7E70020E0E72DE9F3418368074602
:109B1000884623B90026304602B0BDE8F0810DF139
:109B20000701FFF7F5FE06460028F3D09DF8074031
:109B3000220616D504F07F040725BB68002BE9D068
:109B40000DF107013846FFF7E3FE0028E2D09DF84B
:109B5000072002F07F03AB401C43130605F1070505
:109B600002D4C8F80040D6E7232DE6D1D2E773B57A
:109B70000D4601A90446FFF7C7FF064618B900269F
:109B8000304602B070BD94E80F0085E80F000199DF
:109B90008A42F4D3A960A3685B1AA360F0E70000CF
:109BA00030B5044685B01546A9B90268114B9A42F2
:109BB00011D0102D06D82A4669462046FFF7F0FF3F
:109BC00005B030BD102269462046FFF7E9FF0028A6
:109BD000F6D0103DEDE7A368AB4201D20020EFE7DD
:109BE00023682A46204698470028F7D0A3685D1BC3
:109BF000A560E5E75F990700F7B50E4601A907469E
:109C00001546FFF781FFA8B1019A0123D3184FF041
:109C1000000404D2717801F0C001802901D12046EE
:109C200008E031799942FAD329463846FFF7B8FF60
:109C3000019BEC5403B0F0BD73B50D4601A9064677
:109C40001446FFF761FF90B1019AFF2A11D86B7893
:109C500003F0C003802B02F101010AD02B798B4263
:109C600007D32146304601F8012BFFF799FF02B0D8
:109C700070BD0020FBE713B5144669460822FFF7C4
:109C80008FFF18B1DDE90023C4E9002302B010BD45
:109C900013B5144604220DEB0201FFF781FF08B152
:109CA000019B236002B010BD13B5044605291FD8DF
:109CB000DFE801F0030F151E1E1C012201A920463A
:109CC000FFF76EFF18B19DF90430002BF5DB02B0F1
:109CD00010BD082200212046FFF762FFF7E701A927
:109CE000FFF712FF0028F2D0019AF3E70422F1E710
:109CF0000020ECE710B543681A787AB103F10C0242
:109D000042601A7B62B90168C368C0E901128C78AD
:109D10002344036191F903100B444361104620E092
:109D200059781A7901F03004302C1BD15C7B04F097
:109D30003004302C1ED199780269521A0261002237
:109D4000597811F0300F02BF816801318160997B31
:109D5000114402690A44026193F90F301A444261C6
:109D6000012010BD01F0F004202C03D1597911FB22
:109D700002F2E5E701F0C001802908BF0422DFE715
:109D800009B9034B1970034B1B6803B1184770479F
:109D9000C42E0020F82E00201F4B204A1B6800BF55
:109DA00000BF00BF00BF00BF00BF00BF00BF9342A5
:109DB0002FD000BF00BF00BF00BF00BF00BF00BF6B
:109DC00000BF00BF00BF00BF00BF00BF00BF00BF9B
:109DD00000BF00BF00BF00BF00BF00BF00BF00BF8B
:109DE00000BF00BF00BF00BF00BF00BF00BF00BF7B
:109DF00000BF00BF00BF00BF00BF00BF00BF00BF6B
:109E000000BF00BF00BF00BF00BF00BF00BF00BF5A
:109E100000BF0138C3D17047602C00200024F4003B
:109E200018DF70471FB50023CDE90133039368465F
:109E300002230093FFF7F4FF05B05DF804FB000078
:109E4000074A136829B923F00303136043682BB151
:109E5000184723F0010343F00203F6E7704700BF01
:109E600078330020F0B50346186880F308885868F6
:109E7000FF2464B2EFF30585002D01D1A64600470B
:109E80002546064621273FBAF0B4002400250026C7
:109E90000027F0B4F92040B2004700BFF0BD00BF7A
:109EA00013DF7047074A4FF0FF3108B5C2F8801042
:109EB0000346FFF7F5FF20B91846BDE80840FFF755
:109EC000D1BF08BD00E100E0024A1368013B136006
:109ED000704700BF7C33002067DF704763DF704747
:109EE000ADDF7047A9DF7047A8DF7047A6DF704776
:109EF0007FB50023CDF80A30ADF80E3001238DF880
:109F00000A300DF10603ADF80810049302A9044BC2
:109F1000ADF806200593FFF7E9FF07B05DF804FBF5
:109F20008033002010B40D4B024618884FF6FF73A3
:109F300098420FD00A4B1B68DB070BD5094B6024F6
:109F40005A7099701C70084B5DF8044B9989032274
:109F5000FFF7CEBF08205DF8044B7047662C002049
:109F600074330020803300204A33002010B4154B96
:109F7000024618884FF6FF7398421FD0124B1B6899
:109F8000DB071BD5114B60241C7003245C7001247B
:109F90009C70140ADA701C71140C120E9A710A0A61
:109FA000D9711A720A0C090E5A7299725C71084BB7
:109FB0005DF8044B99890B22FFF79ABF08205DF8E2
:109FC000044B7047662C002074330020803300203F
:109FD0004A330020A5DF7047A2DF7047A0DF70473B
:109FE00086DF70477FDF70477DDF70477CDF70471B
:109FF0007ADF704776DF704774DF704773DF704732
:10A0000072DF70476DDF70476CDF704761DF70474C
:10A0100060DF704710DF704748DF70470C4B1B78DC
:10A02000062B10D10B4B1B681A070CD10A4B186872
:10A0300000F0F003302B08D000F0E000A0F1400366
:10A04000584258417047002070470120704700BFB8
:10A05000E00F00F0E40F00F0E80F00F0094B1B7870
:10A06000062B0CD1084B1B681A0708D1074B186840
:10A0700000F0F000A0F13003584258417047002032
:10A08000704700BFE00F00F0E40F00F0E80F00F0B1
:10A09000BFF34F8F0549064BCA6802F4E0621343D1
:10A0A000CB60BFF34F8F00BFFDE700BF00ED00E0C6
:10A0B0000400FA0508B5FFF7EBFF00002DE9F743B0
:10A0C000244E254F33683A68B3FA83F56D09002AA8
:10A0D0003BD0DFF8888098F8003003F0FF046BBBBA
:10A0E00001A8FFF799FF052823D008B1FFF7D0FF9B
:10A0F0003B6801989847F5B9184DDFF86480DFF8A0
:10A1000064902B78D3B9B8F80030ADF80230D9F8A4
:10A1100000300DF102011846FFF778FF052810D036
:10A120000028E3D1326818469047002CE9D1254633
:10A13000CFE70124DFE70125002CCCD003B0BDE838
:10A14000F083002CFAD10124F1E7002BF6D0012492
:10A15000D2E700BFF42E00205434002050340020F9
:10A16000F02E00206C34002008B509B1FFF790FFF5
:10A17000034B1B781BB1BDE80840FFF79FBF08BD2C
:10A180004F34002008B5FFF783FF0000084B5A6EDC
:10A19000013A5A6622B907490A7822F002020A7087
:10A1A0001A6E0132042A08BF00221A66704700BFE7
:10A1B000A43300207033002028DF704729DF704768
:10A1C000082910B501D0FFF763FFD0E90030BDE8E2
:10A1D000104018477BDF704775DF704737B5164B67
:10A1E00018884FF6FF73984210D0144A144D137814
:10A1F000297B0133DBB2994213702C4608D31149F5
:10A20000FFF7EAFF10B1AB6903B1984703B030BD67
:10A21000002313702B7C33B13B21FFF7EBFE10B111
:10A22000AB6903B198476369002BEFD000228DF82A
:10A23000042001A8E9E700BFFE2E002068340020BA
:10A24000002F00209C33002030B53AB11368DB4367
:10A250000A4D0144884204D1D84330BD4FF0FF334A
:10A26000F6E710F8012B5340082213F0010418BF41
:10A270002C46013A84EA5303F7D1EBE72083B8ED8B
:10A2800010B5084B9A685AB150B9EFF3108172B605
:10A29000054A1C6814605C685460986001B962B635
:10A2A000002010BD7434002000E100E01F4B204A64
:10A2B0001B6800BF00BF00BF00BF00BF00BF00BFE2
:10A2C00000BF93422FD000BF00BF00BF00BF00BF40
:10A2D00000BF00BF00BF00BF00BF00BF00BF00BF86
:10A2E00000BF00BF00BF00BF00BF00BF00BF00BF76
:10A2F00000BF00BF00BF00BF00BF00BF00BF00BF66
:10A3000000BF00BF00BF00BF00BF00BF00BF00BF55
:10A3100000BF00BF00BF00BF00BF00BF00BF00BF45
:10A3200000BF00BF00BF0138C3D17047602C0020C0
:10A330000024F40010B50A494A788C78531CDBB22B
:10A340009C4208BF00230C789C421FBF03704868E2
:10A3500002EB420200EBC20008BF002010BD00BFAC
:10A360009033002073B5154E736823B3144D6B6999
:10A370000BB300240DF107002C748DF80740FEF795
:10A38000F9F80DF10600FFF7D5FF90B10223037035
:10A390009DF80630456073709DF80700FFF770FF69
:10A3A00024B9084B4FF48012C3F80021204602B0B4
:10A3B00070BD0424F0E70824F8E700BF90330020C4
:10A3C0001C2F002000E100E010B5114C21684A0765
:10A3D0001BD441F004030F482360FFF7DDFC0E4B54
:10A3E00018884FF6FF73984204D01321FFF702FE3E
:10A3F00048B110BD8B0706D5FFF7FEFD0028F8D148
:10A4000041F006012160FFF7ADFF0020F1E700BF3A
:10A4100074330020C0D40100662C00202DE9F347DE
:10A42000334B344A5B881188334DDFF8E080994222
:10A430000BD852889A4208D36B69002B56D100235F
:10A4400088F8003002B0BDE8F08798F800403CB1D1
:10A450006B69002BF3D000228DF8042001A841E0A5
:10A46000264ADFF8AC901278D5E90163002A18BFBC
:10A470001E46D9F80430002B36D0042E2DD9204F9B
:10A480007B698BB37B7C8DF80440012B01A80CBF4A
:10A49000B2464FF0000AFEF76DF80DF10300FFF72A
:10A4A00049FFC0B101230370164B4760D3F8043550
:10A4B000C0E904A4C0E902369DF8033089F80130F0
:10A4C0009DF80400FFF7DCFE44B90F4B4FF48012F7
:10A4D000C3F80021B3E70424F2E70724AB69002B9B
:10A4E000ADD020469847AAE70824F7E70122B3E752
:10A4F0003C2F00209C330020002F002068340020D7
:10A500001C2F00200010014000E100E0FC2E002084
:10A51000903300200D4B0E494FF4003210B5C3F8B4
:10A52000802001244FF48033C1F848332F20C1F834
:10A5300008334C60FFF7BAFE064B8C602F200021D9
:10A540001960FFF7B3FE044B197010BD00E100E085
:10A5500000100140643400204E340020F8B5124C45
:10A56000124D264622782B789A4200D1F8BD2378E6
:10A570000F48104A078812680F48DBB219B202EB85
:10A58000C10C006852F83120BCF8041003FB07002E
:10A5900090470A4A23781288DBB29A4286BF013379
:10A5A000DBB200233370DDE71C3400200C340020C4
:10A5B0001834002014340020103400201A340020F5
:10A5C00038B5064C064D636E042B00D038BD2846C6
:10A5D000FFF7E2FBFFF7C2FFF5E700BFA43300205F
:10A5E000A08601005B689A68054B9A4206D1D0E9C3
:10A5F000012304490132013B0A604B60704700BFF0
:10A6000068CD0700E82E002008B5084E084CA41BB2
:10A61000E40800250436AC4203D056F8353098479C
:10A6200008B1FFF735FD0135F5E700BF802C0020AC
:10A63000882C00204FF0A043D3F81005C0F38070A1
:10A640007047000070B543F208031C68164B196888
:10A65000A1F54051091B814224D3144B144E1D6AAD
:10A660003460012D1AD19A6902F6FF7222F47F62DA
:10A6700022F00F02891A88424FF0000103D9C3E982
:10A680000451183304E02244C3E904153260243332
:10A690000022C3E901221860104670BD0022C3E900
:10A6A0000422EEE70420F8E714100010AC35002077
:10A6B0006C33002070B59CB000230022109300235F
:10A6C000CDE912234C4B4D4A4D4C4E4DCDE9142350
:10A6D0004D4BCDE916434D4BCDE918534C4B1A93D6
:10A6E00003F17453A3F52303A3F692431B9309B11B
:10A6F000002852D0044645180026A54250D1454DA9
:10A700002C68002C49D0109A1CA9531C372A0A44E3
:10A710004FF0800102F8701C4FF0000260D8382B17
:10A7200057D1DDE9122310980821E1FB00231046E0
:10A73000194612BACDE912010F9269461A0A8DF82C
:10A740003B308DF83A2008461A0C1B0E8DF8392044
:10A750008DF83830FDF734FF621E00231B99D94075
:10A7600002F8011F1A99D94011711999D940117233
:10A770001899D94011731799D94011741699D94075
:10A7800011751599D94011761499D9400833202BA9
:10A790001177E3D16B60002000E00E201CB070BD8B
:10A7A000109B14F8011B1CAA1A440133402B02F819
:10A7B000701C1093A1D169466846FDF701FF129BFA
:10A7C000139A109613F5007342F10002CDE912328C
:10A7D00093E70DF803200133A1E70DF803200133BF
:10A7E0003F2BFAD969466846FDF7EAFE3822002178
:10A7F0006846FDF797FE94E785AE67BB67E6096A92
:10A8000072F36E3C7F520E513AF54FA58C68059B52
:10A81000ABD9831FE82E0020044A00230360436065
:10A820008360C2E90C33C2E904337047AC350020C1
:10A8300030B5264D2C6814F002018BB044D11022A3
:10A8400001A8FDF76FFE0B23ADF80230204B0593F6
:10A8500045F60213ADF818300DF10201FE230DF19B
:10A860001D008DF81A30FFF7BFFB18BBBDF80210B2
:10A870000B2921D84B1C8DF81B30092319448DF866
:10A880001C3089B200231A46C9B205A8FFF7B8FBED
:10A8900080B98DF8040002908DF80C002823ADF8E3
:10A8A000100001A8ADF80E30FFF7A8FB10B944F076
:10A8B00002042C600BB030BD0C238DF81B30082334
:10A8C0008DF81C301421DDE70020F3E774330020FD
:10A8D000020106032DE9F04194B04FF404330493D0
:10A8E000FFF7A0FA0446002840F03D81A748FFF793
:10A8F000D7FA0446002840F03681A54BA54A1A60D5
:10A90000A54B50221A80A54BA54A1A60A54A136888
:10A91000C3F340331BB14FF40051C2F88010A24979
:10A9200004A8FFF777FB9F4A28B113B14FF40053F7
:10A930001360FFF7ADFB9D4B0121197092F81633A0
:10A940005806F6D59A4B9968002900F010811A68CC
:10A9500042F480021A60162200210DF13600FDF744
:10A96000E1FD0022139240F20112ADF83C201722C3
:10A97000ADF844208F4A01920123019A089208A958
:10A980000DA8ADF834308DF83E30FFF741FB019A49
:10A990000446002840F0E780874A88491160CDE9E5
:10A9A0000D00112208A88DF81020FFF72BFB04469C
:10A9B000002840F0D8809DF8212008A801328DF8A9
:10A9C0002120FFF721FB0446002840F0CC8007221D
:10A9D0007B4904A8FFF70AFB0446002840F0C38027
:10A9E00078494FF0C8720DA8CDE90D12FFF700FBB2
:10A9F0000446002840F0B780734A8DF80A304FF6BD
:10AA0000FF7111804FF65962ADF8082002A96F4A14
:10AA10001846FFF7E3FA0446002840F0A4806C4B88
:10AA200004AC03F1100518685968224603C20833C4
:10AA3000AB421446F7D1654D04A8A91CFFF74EFAA6
:10AA40000446002840F08F8001461C220DA8FDF727
:10AA500069FD9DF83430ADF8004043F004038DF8F3
:10AA60003430AB788DF80E300223ADF80C3014235F
:10AA7000CDE90A44ADF82C302B460C94274604F05F
:10AA8000F80444F003044FF0110803AE08AA0DA91E
:10AA900033F8040B8DF802408DF801800896CDF84C
:10AAA00024D0FFF799FA044600285CD101461C2205
:10AAB0000DA8FDF737FD9DF83430ADF8004023F0C8
:10AAC000180343F018038DF83430AB788DF80E304E
:10AAD0000123ADF80C3007F0E80343F013038DF8C1
:10AAE00002301723CDE90A44ADF82C302B4608AAD2
:10AAF0000DA933F80C0B0C948DF801800896CDF855
:10AB000024D0FFF769FA044668BB324A324D136815
:10AB100043F001031360014618220DA8FDF702FD62
:10AB200040F6CD424FF48043CDE90E2303238DF848
:10AB300040302A4B13930DAC0FCC0FC594E807009F
:10AB4000274B85E8070027481F70FFF743FB0446A3
:10AB500048B9254B4FF6FF721A80244B1F70244BC7
:10AB60005B6843B90824204614B0BDE8F0814FF477
:10AB700080031360EFE61F4B1A7C002AF2D11E4AB5
:10AB80005F745A61FFF754FE0446ECE7008007004B
:10AB90006C3400206C2E0020F02E00206433002046
:10ABA00045B7070000E100E085A107004F34002011
:10ABB00074340020002C0020F42E002055B707002C
:10ABC0005CCC07000C001800662C00204A330020E3
:10ABD00028CC070074330020002F0020B5A0070008
:10ABE000FC2E00209C330020FE2E00206834002024
:10ABF000903300201C2F0020DDA1070010B50C4968
:10AC00004A6E042A044611D00B6E1344032B02F142
:10AC100001024A6688BF043B182202FB0313184650
:10AC20000021FDF77FFC2060012010BD0020FCE723
:10AC3000A433002030B5044685B00D461022002113
:10AC40006846FDF76FFC237A012B0AD0022B0ED049
:10AC500063680193236829469B686846984705B056
:10AC600030BD23690293A38AADF80C30F0E70123CD
:10AC7000A2898DF80030E389ADF80A20D31AADF827
:10AC80000830E5E738B51C4B5A6E19465AB31C6EAE
:10AC9000182202FB04331A7A012A07D0022A23D091
:10ACA00018460921BDE83840FFF7C4BF1825D88AE7
:10ACB0009A8A05FB0414D4E90314121AB2F5806FC2
:10ACC0004FEA80000144B4BF92B24FF48062204446
:10ACD000FFF774FA11280BD1084A137823F0020306
:10ACE00043F00403137038BD9889FFF765FAF1E764
:10ACF0000028F8D0D4E700BFA43300207033002030
:10AD000038B52A4A13780146980742D5284A146E66
:10AD10001820022900FB042005D003292DD0BDE80E
:10AD20003840FFF7AFBF234B00211970037A012B86
:10AD30000CD0022BF3D18389028A01338381C3892A
:10AD400001339BB29A42C381E9D111E0858AC38A5B
:10AD5000E91AB1F5806FB4BF89B24FF480610B443A
:10AD600018219BB201FB04229D42D382D7D100213E
:10AD7000FFF760FFFFF70AFAD1E70E4A13780133B5
:10AD8000DBB2032B01D81370C9E70023137008212D
:10AD9000EEE75907C3D50649496E03F0FB0313706C
:10ADA0000029BCD043F00203EDE700BF7033002060
:10ADB000A43300204C340020054A137813F0060F0A
:10ADC00004D143F002031370FFF75CBF704700BF6C
:10ADD000703300202DE9F043494ED6F8009019F069
:10ADE000040F85B0054614464DD019F0020F40F00F
:10ADF000818049F001033360424B1B78DB073CD56F
:10AE0000414F424B9F423AD3414B9F4237D2002899
:10AE100037D0C0F30B0373BB3B68984204D20520C4
:10AE200029F0010333601FE08AB27B6800EB023235
:10AE30009342F4D31FFA81F8B8F1000F19D0684695
:10AE4000FFF7DCFE98B1009BC3E90074009B02226F
:10AE50002D0B1A729D81A3F81080FFF7ADFF3368A8
:10AE600043F001033360002005B0BDE8F083072004
:10AE7000D6E70420D4E70620D2E70120D0E702205D
:10AE8000CEE70320CCE7C0F30B03ABBB214E0F464C
:10AE90004FF0020C3246C6F804C5D2F800E4BEF109
:10AEA000000FFAD0C2F80805D2F800E4BEF1000F96
:10AEB000FAD0C2F80435D6F800E4BEF1000FFAD09B
:10AEC000013F00F58050E6D105EB0136B4B13946BB
:10AED00010226846FDF726FB310B01232D0BADF840
:10AEE0000A10684639468DF800300194ADF80850D4
:10AEF000A047B8E70A20B7E70620B5E72046B3E742
:10AF00007833002070330020702C0020702C00203B
:10AF1000802C002000E001402DE9F0430F46464917
:10AF20001C460B6813F0040F85B00546884646D0D2
:10AF30009E0777D443F001030B60404B1B78D80782
:10AF400072D53F4E3F4B9E4270D33F4B9E426DD2D7
:10AF50001FB9032005B0BDE8F083002DF9D047EA02
:10AF60000503990701D00620F4E733689D425FD3BB
:10AF700093B2716805EB8303994259D31FFA82F9A2
:10AF8000B9F1000F01D10420E4E76846FFF736FE6F
:10AF900098B1009BC3E90064009B01221A72C3E9C7
:10AFA0000375A3F81490FFF707FFD8F8003043F0BB
:10AFB0000103C8F800300020CCE70720CAE7002FC3
:10AFC000C7D00028C5D047EA00039B07CBD1002A91
:10AFD000D9D01E4B0121C3F80415D3F80014002961
:10AFE000FBD01A490023084657F8236045F8236030
:10AFF000D1F80064002EFBD001339A42F4D1002333
:10B00000C1F80435D0F80034002BFBD000268CB1F9
:10B01000314668468DF80060CDE90145ADF80C2059
:10B02000A047C8E70A2095E7012093E7022091E7AF
:10B0300005208FE720468DE778330020703300200D
:10B04000702C0020702C0020802C002000E001409B
:10B05000F8B51E4C1E4F0646254623789BB90123A2
:10B0600023701C4B1C4C1E60FFF7AAFA0022012122
:10B070002046FFF7AFFE07280246F5D048B100236F
:10B080002B700320F8BD3846FEF786FEFFF766FA00
:10B09000E3E7124C124F134E5821201DFFF7D4F84E
:10B0A000214620604FF4AE720E480B4C01F0A0FD1B
:10B0B000FFF786FA3B46572231462046FFF72CFF22
:10B0C0000728F5D00028DDD0D9E700BFC42E002026
:10B0D000A0860100F82E002000F00700AC3500200B
:10B0E000819D0700583700202DE9F04F1E4E1F4963
:10B0F000726B336B02F6FF74E41A0C40A50805F678
:10B10000FF7585B003F580570D4003EB00080AB1C9
:10B11000934226D04FEA95094FF0010A4FF0030BF6
:10B120006846CDE900A8CDE90279FEF779FEA8B915
:10B130006846CDE900B7CDE90289FEF771FE68B92E
:10B14000A542736B8CBF0446641B1B1B00202F445D
:10B15000A8443363FFF77CFF002CE1D105B0BDE8C4
:10B16000F08F0020FAE700BFAC35002000F0FFFFB1
:10B170007FB5124B0C685B6B1D18E41A0323009318
:10B180000F4BA4086846CDE901350394FEF748FE4D
:10B19000064638B90846FFF73FFB3046FFF758FF31
:10B1A00004B070BD102200216846FDF7BBF9684667
:10B1B000CDE90154FEF734FEF2E700BFAC350020C4
:10B1C0000080070030B54268527802F00F0108296C
:10B1D00087B003460FD103691C6800250CB907B07E
:10B1E00030BD214625736846FEF79CFB6846FFF795
:10B1F000E9FFA468F2E712F0C00120D102F03000AC
:10B2000010280ED15A6911705A68186953789468D9
:10B2100003F00F03072B09D10146204600F017F871
:10B22000DDE79006F0D55B691970D8E71279214601
:10B2300014B101F0DDFCD2E7FDF774F9CFE7802906
:10B24000CDD10069002192060160C8D5EBE77FB53A
:10B250000023CDE902318378194490F90330049139
:10B26000194403780591CDE900003BB16846FFF72A
:10B27000A9FF6846FEF73EFD0028F7D107B05DF84C
:10B2800004FB00002DE9F04355686B7813F0C0040F
:10B2900089B006468C46174603D0402C6AD000245D
:10B2A0000AE003F00F025E4903F03003102B51F85F
:10B2B000228020D004D8CBB1204609B0BDE8F0836D
:10B2C000202B1ED0302BF7D17B6929781970072AE3
:10B2D0000AD17B6838691A792146FDF723F97B6822
:10B2E00039699868FFF7B3FF3A6940E03A6929463F
:10B2F000C0470446E0E77B6901221A703A69796821
:10B30000F6E7BCF1020FD7F8149024D1042A22D812
:10B3100004A9FEF72CFC04460028C0D0069B2BB1E4
:10B32000796899F800304A799A4205D8059B73608C
:10B33000069B002BC0D0B2E708793A6900FB0322D4
:10B3400004A8C04728B199F80030013389F80030CB
:10B35000E4E70446EAE799F800306A799A429ED910
:10B360003A692979581C89F8000001FB03227968A1
:10B370003046BDE7D2F81080454655F8043B13B976
:10B38000FEF792FCB5E7022914D104A9FEF7EFFB02
:10B39000002884D0D8F8003079682A4604A8984755
:10B3A000044600283FF47BAF069B002BF2D1059B9F
:10B3B000736081E701292BD04CB24CB105297FF491
:10B3C0006EAF04220DEB0201FEF7EAFB042424E039
:10B3D0000DF1040901340B2C3FF461AF0122494601
:10B3E0003046FEF7DDFB00283FF459AF19F9013B69
:10B3F000002BEFDB0B4B049301ABCDE905340023AD
:10B400000793D8F8003079682A4604A8984770E76F
:10B41000082201A9FEF7C4FB08240028EAD13EE770
:10B4200038CC07005F9907002DE9F04F8B788FB07B
:10B430000025CDE904521A4491F903300692CDE972
:10B440000055CDE902111A44044607924FF0010855
:10B45000A3682BBBDDE9033402A85D78FEF74AFC44
:10B460000028F7D115F0300F03D1039B1B7803B1EF
:10B470000134002C65D06309002293425BD10EAAEF
:10B4800002EB830304F01F044FF0FF30C4F12004EB
:10B4900020FA04F453F8380C231A5842584108E0B3
:10B4A00008A92046FEF730FB30B9A368002BD1D0A5
:10B4B00000200FB0BDE8F08F089EDDF80CA0002E34
:10B4C000C8D0F70806F00706039B1A78974204D104
:10B4D0005B7803F00F02082A58D102A8FEF70AFC95
:10B4E000DDF80C90CA45EFD1BD420DD8039A5378D0
:10B4F00003F00F03082B29D002A8FEF7FBFB039BE8
:10B500009945F3D14FF0FF3531462046FEF7CCFB8D
:10B5100000289DD1CCE79B681B789F4233D14946D8
:10B5200008A8FEF7FFF989F80C8008AA31462046E2
:10B53000FFF7A8FE25E05DF822100131B8D10132F5
:10B540009BE70120B5E79A45DED081E71578BD423B
:10B55000DAD8069BD4F808A0D3F80090A368B9F114
:10B56000000FF0D09A457FF473AFD9F80030D3F8CC
:10B5700000B0BBF1000FCED033463A4649462046D4
:10B58000D847002894D0D9F80890E7E713F0300F97
:10B590000FD1049B3F2B0CD85A090EA901EB820254
:10B5A00003F01F0352F8381C08FA03F30B4342F868
:10B5B000383CD4F80C90B9F1000F04D002AB3246FD
:10B5C00039462046C84702AA31462046FFF75AFEB0
:10B5D0009EE7F0B585B00E468C686946074615466D
:10B5E000FEF7C5FA88B1B06878B1737803F030031C
:10B5F000202B03D129462046FFF729FE2A46214663
:10B600006846FFF711FF019B7B6005B0F0BD0000AD
:10B6100070B50D4B0D4C9A6B0D4E0E4D0E492160C1
:10B620005C33C4E901320D4BE3600D4B002231461F
:10B630002846C3E90022FFF70AFE32462946204683
:10B64000FFF7F2FE70BD00BFAC3500204837002088
:10B6500080340020E4CD07005F990700E5A50700CE
:10B66000E82E00202DE9F341002406460DF10700E5
:10B670000D4617468DF80740FCF77CFF204B214A0A
:10B6800018781178CBB2204909888B4238BF013332
:10B69000C0B238BFDCB2A04228D014781378DBB235
:10B6A000994286BF0133DBB2002313709DF8070077
:10B6B000FEF7E6FD4FF6FF739C421ED0134B1B684E
:10B6C00003EBC40843F834709EB195B1104B188851
:10B6D000104B1B682A46314604FB003001F088FA03
:10B6E000A8F80450002002B0BDE8F0814FF6FF74C6
:10B6F000DCE70020A8F80400F5E70420F3E700BF2A
:10B700001C3400200C3400201A3400201434002093
:10B71000183400201034002007B5084B1B88072B75
:10B72000CDE9000107D9064A08216846FFF79AFFCC
:10B7300003B05DF804FB0920FAE700BF18340020CD
:10B74000C1A107000021024A0846FFF78BBF00BFD6
:10B7500069A107002DE9F04F0388112B8DB0044635
:10B7600039D010D8102B23D02388142B00F08D83D0
:10B7700057D8102B00F0B08045D8022B00F0BF80C6
:10B780000DB0BDE8F08F122B36D0502BECD1A54D6B
:10B79000C288EB899A42E7D1038A022BE4D1837CE9
:10B7A000D90715D4FEF7DEFD0028DDD0AB691FE018
:10B7B0009D4B82881A8000F1100303CB9B4A9C4B5F
:10B7C0001060516000221A70964BDB89002BCBD1A0
:10B7D000FEF724FEC8E7944B4FF6FF721A80944B95
:10B7E00000221A70FEF7BEFD0028BDD08D4B9B696C
:10B7F000002BB9D09847B7E700F1080303CB8B4A79
:10B8000010605160E4E7112B6FD0132BB8D1894839
:10B8100000231A4685210088FEF7E4FB0028AFD0FC
:10B8200066E0522B00F0388346D8502B00F03B8363
:10B83000512BA5D1A579002DA2D01022002108A856
:10B84000FCF770FE022D9BD17B4E2289B3899A4270
:10B8500096D1A37B043B022B92D99DF82630318AE6
:10B8600043F001038DF82630238AADF82830638A2F
:10B87000ADF82A3004F114030B930023ADF81A300D
:10B8800005AB07936B4B1D8802228DF82020ADF885
:10B890001820284606AAFEF79DFB002835D19DF802
:10B8A0001430DA0731D440F2FD1308A92846ADF868
:10B8B0002430FEF719FB63E7552B00F01684562B56
:10B8C0007FF45EAFA379002B7FF45AAF594B13215D
:10B8D0001888FEF78FFBA1E7564BA2881A80574ABB
:10B8E000136823F0020313604AE7FEF7A1FF08B1D3
:10B8F000FEF7CEFB4F4B4FF6FF721A8040E74D4BE1
:10B9000000211888FEF7E8FA88E7002308A92846EE
:10B91000ADF82430FEF7E8FA00287FF431AFCDE926
:10B9200008000A90207D431E052B00F2AC82DFE860
:10B9300013F00600330243029D00AA025902638AF3
:10B94000062B01D0032116E03D4BD4F816501A887F
:10B950003C4B0A951A80637D0993012293428DF82E
:10B9600020200CD1384A1370374B1C78012C0AD098
:10B97000022C1BD005210120FEF7D4FA00E7022B90
:10B98000F0D00721F7E7002DDCD0B5F5807F45D852
:10B990002E4E2F4B00271C22394606F13C001F700B
:10B9A000FCF7C0FD3763B5630121E4E7002DC9D082
:10B9B000C5F30B0333B1254B264A5B6D12682B444C
:10B9C0009342BFD1B5F5805F28D8214B1B783BB39C
:10B9D0001E4B204A586D12682918914220D8DA6C03
:10B9E0001865C3E911521C4A186313781B4C0133C4
:10B9F00003F0030313701A4B00221A802368194ABC
:10BA000001332360184B1B6801211844FFF7E2F94A
:10BA10000028C9D02368013B2360ABE70421AAE7D3
:10BA20000821A8E7002F0020FE2E00203C2F002038
:10BA300068340020662C00204A3300207433002034
:10BA4000983300209A330020642C0020AC3500206D
:10BA50006934002068330020442F00207C3300200C
:10BA600048330020C99E07006C33002003238DF863
:10BA70002030974B1C78012C04D0022C00F0D6808B
:10BA80000524ADE0934FD7E90E21914240F0828129
:10BA9000914E3378002B40F0A380FFF7B9FD0128C9
:10BAA000EED18E4B93F874201C46002A00F0B9802A
:10BAB00093F87A30002BE3D0894DD5E90001A8B185
:10BAC000A1B194F8DB3013B194F8DC3073B994F879
:10BAD00084305BB1D4F88830342B07D194F88CC013
:10BAE000804A002343F20C0E634501DB0A2477E011
:10BAF00052F8049BBEF80080C14500F0FC8201337F
:10BB0000F2E794F87C30002BF0D0BA68D4F880309B
:10BB10009A42EBD894F8E830002BE7D1724B2B60B7
:10BB200020236B60FEF7C6FD0028DFD194F8E97092
:10BB30006E4B6F493A46184601F05AF86D4A402F4D
:10BB40000346C2E900079BD12968002998D011F06B
:10BB5000030795D1684A00926A686848FDF732FC8D
:10BB600000288DD0664D94F8A1302F60032BBDD8EE
:10BB7000DFE803F00C39294194F87C30002BB5D074
:10BB8000FA68D4F880309A42C4D3AFE794F8B03062
:10BB9000002BABD0D4F8B4302B605A4B524C03F18D
:10BBA000200718685968224603C20833BB4214466E
:10BBB000F7D1286880B3FEF745FD80B90124FFF76F
:10BBC00047FA34700CE094F8A830002B8ED0D4F8EB
:10BBD000AC202A604C4BC3F5FC239A42DDD90424E7
:10BBE00021460420C8E694F8A230002B3FF47EAF33
:10BBF000D4F8A430D0E794F8A830002B3FF476AF07
:10BC000094F8A230002B3FF471AFD4F8A430D4F8EC
:10BC1000AC20991829600BB90324E1E7002AD9D197
:10BC2000FAE71B78002B7FF461AF29E7294CD4E9B0
:10BC30001423616CD31A9942264640F0AB80A36C62
:10BC400062650020E3646064FFF702FA2C4B216D0B
:10BC50001A689142984632D12C4C2368002B30D17F
:10BC60001E4D95F8B930032B2ED11D4F1E4B3B6056
:10BC7000274BD8F8001018684FF02009C7F8049037
:10BC8000FEF718FD4A46002805F1BB01386814BFCD
:10BC90000A24012400F09EFF002818BF05247369C0
:10BCA000A3B1012B7FF422AF1A4B012C6ED195F872
:10BCB000A120032A68D8DFE802F031555B61012436
:10BCC0008EE7FEF74BFCC8E70A24E8E7124BECE7E7
:10BCD000642C0020AC350020693400208034002022
:10BCE000E82E002010350020C82E00200837002044
:10BCF0006A350020BC2E002064CC070050CF07001E
:10BD0000683300203B350020008007007C33002092
:10BD10006C330020D0350020C435002001229A6009
:10BD2000D5F88020B260B26C5A60D8F800201A6052
:10BD300000212022B248B34DFCF7F4FBB222FF21D0
:10BD4000B148FCF7EFFB00233363B04E2846FFF702
:10BD50007FF911287FF444AF3046FEF71DF8FEF757
:10BD6000FDFBF3E7A5229A60D5F8A4207263DAE719
:10BD7000AA229A60D5F88020F260D4E7AC229A60BB
:10BD8000D5F8A4207263F5E70A24CCE70022C3E9C2
:10BD90000122CCE7082423E7638A032B02D0032186
:10BDA0000220E9E5A27D637D43EA0223984A1380DD
:10BDB000984A01211380F3E704238DF82030964B35
:10BDC0001B78012B04D0022B08D005210320D3E5DA
:10BDD000924BD3E90F01FEF7C9F8D1E48F4B186DF0
:10BDE000996CF8E7638A022B02D003210620C3E591
:10BDF000637D09930622012B8DF8202009D1864A04
:10BE00001370854B1B78012B07D0022B35D00521F1
:10BE1000ECE7022BF3D00721E8E7804BD3E90F12C0
:10BE20004FF480704FF6FF739D423FF4A9AC7C4BFA
:10BE30001B68DB077FF5A4AC7A4B000A60241871FD
:10BE4000080A1C70D97106241872080C090E5C705F
:10BE500099720124110A9C70DA7200241973110C72
:10BE6000120E587259739A73DC705C719C710F22B8
:10BE7000B1892846FEF73CF882E4684B4FF48050C5
:10BE80009A6C196DCEE7032176E500231A46194610
:10BE9000A088FEF7A5F8C1E400231A461946A08839
:10BEA000FEF720F8BAE4604BE2889B889A427FF460
:10BEB00067AC0223002508958DF82030564B268A62
:10BEC0001B780A9604F11207012B099715D0022B53
:10BED00032D0AA464E4B1E88002E3FF451AC4D4C3A
:10BEE0002388013B9BB22380002B7FF449AC294679
:10BEF0005046FEF73BF8268042E4484CD4F83CA07C
:10BF0000A36B06EB0A029A4201D9256CE2E70AF11B
:10BF10005C0032463946204400F06AFEE06B04F1D2
:10BF2000400206EB000A31463846C4F83CA0FEF752
:10BF30008BF905462064CDE73C4B384C1B78D4F890
:10BF400050A0A56C002BC5D0B6F5807FC2D8636D1C
:10BF5000626C06EB0A09A9EB03039342BAD804F119
:10BF6000480231463846FEF76FF93149DFF8C8A07C
:10BF70000B78BAF80020A0644FEA032B2D4BC4F8CD
:10BF8000509005460BEB02001844B318FF2B0393A7
:10BF9000884659D83246394600F02AFE039BAAF853
:10BFA0000030CA46244E3288002A93D0636D206B3D
:10BFB000616CD31A03448B428CD3204B204FD3F8AF
:10BFC00000C03B6898F800E01A49013303323B6037
:10BFD00092081C4B01EB0E216044FEF79DFF0028E8
:10BFE00079D1236B32881344236398F800300133EE
:10BFF00003F0030388F80030002333806AE700BFB2
:10C00000E435002009A6070008360020A0860100BC
:10C01000983300209A330020642C0020AC35002097
:10C0200074330020803300204A330020693400201C
:10C03000442F0020482F0020483300206C3300207C
:10C040007C330020C99E0700C2F580739BB21A465C
:10C050003946039300F0CCFD039B206B2E49F61A62
:10C060001F440A962D4B2E4E09971F6833684FF4D4
:10C0700080720133AAF8002033604022294B5944D2
:10C080003844FEF749FFE0B9BAF80020236B1344A7
:10C090002363CA4698F80030234F0A9E013303F009
:10C0A0000303002288F800303A80002E3FF47AAF74
:10C0B00019480999324600EB032000F099FD3E80B3
:10C0C00070E73368E56CD4F854A0A564013B336095
:10C0D000C4F850A0DEE73B68E56CD4F854A0A56432
:10C0E000013B3B60C4F850A07FE71721A088FDF713
:10C0F000F7FEFFF793BB94F8A120032A3FF6F6ACB6
:10C1000001A353F822F000BF03BB070015BB0700D3
:10C1100079BB070079BB0700482F00206C33002053
:10C120007C330020C99E07004833002008B5074B28
:10C130001B681BB1984740B1FDF7AAFF044B1B7861
:10C140001BB1BDE80840FDF7B9BF08BD643300204E
:10C150004F34002008B5FDF781FF10B1774B784AC6
:10C160001A60FDF75BFF28B1764B774A1B68C3F373
:10C1700042331360FDF772FF20B1744AD36823F095
:10C180008073D360FDF74AFF40B14FF08043002237
:10C19000C3F80C21C3F81021C3F83825FDF75EFF62
:10C1A00010B16B4B03221A60FDF758FF40B1694B89
:10C1B00005221A6001229A6700229A603F225A6083
:10C1C000654B1B78062B50D1644B1B6819074CD16B
:10C1D000634B1B6803F0F003502B46D14FF08052A5
:10C1E000604BD2F80414C3F82015D2F80814C3F831
:10C1F0002415D2F80C14C3F82815D2F81014C3F87B
:10C200002C15D2F81414C3F83015D2F81814C3F84A
:10C210003415D2F81C14C3F84015D2F82014C3F812
:10C220004415D2F82414C3F84815D2F82814C3F8DA
:10C230004C15D2F82C14C3F85015D2F83014C3F8AA
:10C240005415D2F83414C3F86015D2F83814C3F872
:10C250006415D2F83C14C3F86815D2F84014C3F83A
:10C260006C15D2F84424C3F87025FDF7D7FE28B129
:10C270003D4B3E4A1B6803F04F0313603C4AD2F823
:10C28000883043F47003C2F88830BFF34F8FBFF398
:10C290006F8F4FF01023D3F80C22D2071ED5354BE9
:10C2A0000122C3F80425D3F80024002AFBD04FF064
:10C2B0001022D2F80C3223F00103C2F80C322D4BBD
:10C2C0001A46D3F800140029FBD00021C3F8041546
:10C2D000D2F80034002BFBD0FDF7DAFED3F80022B1
:10C2E000002A03DBD3F80432002B23DA214B01228E
:10C2F000C3F80425D3F80024002AFBD04FF0102205
:10C300001521C2F80012D3F80024002AFBD04FF008
:10C3100010231522C3F80422164B1A46D3F8001432
:10C320000029FBD00021C3F80415D2F80034002BFB
:10C33000FBD0D1E7104B114A1A6008BD74C007400A
:10C340000DF0ADBA440200103C050040F0ED00E0F5
:10C35000A005004010560040E00F00F0E40F00F090
:10C36000E80F00F000C0004058020010E40E00404A
:10C3700000ED00E000E00140602C00200090D003C0
:10C3800073B500230DF102008DF80230FCF7F2F8CE
:10C39000264B1B7803F0FF04002B41D1244B1A6875
:10C3A000002A3DD0234AD2F80813C90738D51C60AB
:10C3B0001B68214D01930DF10300019BD2F8086524
:10C3C0008DF80340FCF7D6F86A6829681F2A98BFE1
:10C3D000541CA142F6B26C6004D1202C14BF611C25
:10C3E0000021296015499DF803008E542A68944263
:10C3F0003ABFC2F121021319A31AAA689A4238BFA0
:10C40000AB60FDF73DFF6B682A681F2B94BF0133BB
:10C4100000239A4201BF074A0123C2F80833536040
:10C420009DF80200FDF72CFF02B070BD4F340020D4
:10C4300000D1004000D00040403400201D340020D6
:10C440002DE9F04FAF49B04AB0480B68007887B08B
:10C4500004931378984200F0B0800133DBB2022BD2
:10C4600008BF002313701278A94B53F82240049B95
:10C47000234423F07F430B6001230193A54AA64880
:10C480001378D0F800C050780390506892780592E5
:10C49000A24A02900020D1F8009092F8008019463C
:10C4A000624686468246039DA94240F08980BEF1DD
:10C4B000000F05D0994981F800809249C1F8009099
:10C4C000954900B10A6001980A68002840F0C980C7
:10C4D000BCEB020218BF0122019200268F4AD1F85C
:10C4E00000A012780492874A4FF0000CD2F8009016
:10C4F000504661464FF0010BE646002E40F0B680F4
:10C50000039A9A4240F0D18009B1824B1A70824B53
:10C51000BCF1000F00D018601B689A4502D1019A47
:10C52000002A44D0002B00F01A81D3F800907C4CF4
:10C53000744BD4F8046519687A4F751A3B7825F066
:10C540007F450335A3B94FF48033C4F84433C4F8AE
:10C550000433754B4FF400324FF00108C3F88021CB
:10C560002F201A60C4F80080FDF7A0FE87F8008035
:10C57000A9452CBF4944491921F07F41C4F8401511
:10C58000D4F804359B1B23F07F43891B033321F030
:10C590007F418B420BD9D4F80435C4F840352F20A5
:10C5A000FDF784FE604B4FF40032C3F800215B4B73
:10C5B00000221A7007B0BDE8F08F002401945DE7F7
:10C5C000029E01EB410506EBC5070131059EC9B28C
:10C5D000B14208BF0021029E16F83550022D0AD044
:10C5E000032D7FF460AF002A3FF45DAF82F810A006
:10C5F0000120D269F7E7D7F804B015461646002D9A
:10C600003FF451AFAB4500F0AD802E46ED69F6E743
:10C610000120B4E0D2F800C0A44505D905B10A60F4
:10C62000ACEB0404146059E7A4EB0C046044D2F8AA
:10C630000CC0C2F800E0D2F81C80BCF1000F07D09B
:10C64000049DD661054425F07F45C2E9015C16468C
:10C6500001254246002ADDD1002D3FF43FAF0A609C
:10C660003CE700252E462846AE46F3E73246F669FB
:10C67000D2F804802D4C9768A8EB090525F07F457A
:10C68000A54234D83D441560C2E901EE82F810B0ED
:10C69000C2F81CE030B115680468A5425AD8651B81
:10C6A0000560D0614FF0010C52E0029903EB4302A8
:10C6B00001EBC20401330599DBB2994208BF0023A4
:10C6C000029911F83210012947D16268157C002DBA
:10C6D0007FF416AFA7685760E76897602769D7604F
:10C6E00064699461049C002CC2D05560C0E7A9EB3A
:10C6F000080424F07F44BC423ABF3C1B1460C2F8DB
:10C7000000E0C1E764340020603400206134002080
:10C710005834002090330020703400204D34002025
:10C72000001001404E34002000E100E0FEFF7F00D9
:10C73000ED1BE769A0463FB13C462768AF42F7D3FF
:10C740007F1B2760274644461560D761E261024699
:10C750001046D2E680460446EFE70121D0E6FDF719
:10C76000D9FE24E7B5420AD1D269002A7FF450AF3E
:10C7700008480127876091463846BE46B846D5F836
:10C7800000B0ED69F561002D3FF48DAE2E685E447A
:10C790002E6088E6001001402DE9F8432649274B1A
:10C7A0000025C1F84051C1F84451C1F84851C1F8C1
:10C7B0004C51C1F80051C1F804511B68002B39D00D
:10C7C000D1F804451E49DFF88C800968641A24F00A
:10C7D0007F442F461A68A24217D8A41A15441A7C1F
:10C7E000DE6982B1D8F800901F74D3E90521B9F150
:10C7F000000F06D01046C84728B1FDF749FC334664
:10C80000E8E708469047002EF9D10E4A0E4B117802
:10C810001B788B4205D10133DBB2022B08BF00230A
:10C8200013701278094B43F82250094B4FF48012D1
:10C83000C3F80021BDE8F8830010014070340020E7
:10C84000643400206134002060340020583400201B
:10C8500000E100E0603300202DE9F0474FF0A043F5
:10C860000422AE4CC3F8782786B0AD4BAD49002505
:10C870004FF4AE7220468DF807501D7000F0B8F9E5
:10C880002668721C06D02A465821201DFDF7DCFCC4
:10C8900086420DD04FF4AE720021A048FBF742FE55
:10C8A000012300206360FEF7D3FB08B1FDF7F0FB26
:10C8B00043F208031E682369012B19D06369BBB1D9
:10C8C000A569994F05F6FF7525F47F6525F00F05DD
:10C8D0003544BB68A52B78D00DD8012B1AD0FDF7B5
:10C8E000A9FE0146002800F08F8040F6B83586E0AA
:10C8F00035468E4FEDE7AA2B77D0AC2BEFD12846EB
:10C90000FEF7F2FB064600286BD139462846FEF7B3
:10C910002FFC65E06369012BE1D1276BD4F82490EB
:10C920003E444FF0030AA9EB0707B7F5805F4FF0CD
:10C9300000024FF001013046B84628BF4FF480583E
:10C94000FEF748FA034618B101238DF80730C6E711
:10C95000424629463046FEF7DFFA0028F4D14FEA76
:10C96000980302A8CDE902A604950593FDF758FAAD
:10C9700002460028E8D101212846FEF72BFA0028BC
:10C98000E2D1236B43442363FEF762FBB7EB080756
:10C9900046444544C9D143F208033A46186849461B
:10C9A000FDF752FCA36A984204BF0123C4E90703C0
:10C9B0005D4808BFC4F81890FDF72EFF0020FEF771
:10C9C00047FB0646002EBFD189E72846FEF78CFBC1
:10C9D000064630B93846FDF71FFF3046FEF738FBF4
:10C9E00006460123CDF80730ECE739462846FEF726
:10C9F000BFFBE6E740F2E730FDF758FC013DFDF7ED
:10CA000019FE90B1002DF5D1236A012B7AD8E56982
:10CA1000002D79D043F20803A16918680022FDF7C0
:10CA200013FC2B1A5942594104E0002DECD001238C
:10CA30008DF807309DF8073013B9002940F0B48015
:10CA4000FDF768FD3A4B3B4A1A603B4A3B4F3C4E70
:10CA50000521002591703B49158051603A4A1560C7
:10CA60003A4A15703A4A15703A4A4FF48011E0205C
:10CA7000C2F8801182F81403116001F18041A1F520
:10CA80006F21F61BC1F8085582F81103324AD1F81C
:10CA9000041511603149324A0A603249A8320A60ED
:10CAA000314A1570314A1570314A08211180314AD6
:10CAB00014211180F608AE4228D12F4A137843F092
:10CAC000010313702D4B2E4A1A602E4B04221A605C
:10CAD0002D4B00221A60A36B8BB1FEF799FD70B14C
:10CAE000236A002B56D1A369002B53D0274A136029
:10CAF000264B1868FDF7A6FD254B01221A70FDF79D
:10CB00002DFDFCE7002195E7012193E757F835302B
:10CB1000984700287FF4CAAE0135CCE7AC35002039
:10CB2000C42E002000F00700D0350020C4350020BE
:10CB30006033002019B7070090330020802C0020BC
:10CB4000882C0020F42D0020703400206034002058
:10CB50006134002000E100E064340020143400203F
:10CB6000A42C0020103400200C3400201C340020A1
:10CB7000183400201A340020703300205434002070
:10CB800001AD0700783300207C330020683300209B
:10CB900069340020E36A002BB1D1A369002BAED029
:10CBA0000B4B626A1A60A3E743F208042168FDF7A1
:10CBB00039F910B90846FDF775F92268FDF732F921
:10CBC00010B91046FDF76EF9002006B0BDE8F087F9
:10CBD0006833002030B501390024A24201D1002081
:10CBE00005E0035D01340D5DAB42F6D0581B30BD4E
:10CBF0000A44914200F1FF3300D1704710B511F89B
:10CC0000014B03F8014F9142F9D110BDF8B500BFB7
:10CC1000F8BC08BC9E467047F8B500BFF8BC08BC1D
:10CC20009E467047002C002050EADA308883B89F77
:10CC3000604F15F30000C98EAF9A0700539A0700A2
:10CC4000E1990700919C0700779C0700399C070039
:10CC5000F99B0700D3B50700000000004466755437
:10CC60006172670008200001FFFFFFFFFFFFFFFF69
:10CC7000FFFFFFFF000000000000000000000000B8
:10CC800001000000FFFFFFFF512563FCC2CAB9F39A
:10CC9000849E17A7ADFAE6BCFFFFFFFFFFFFFFFF73
:10CCA00000000000FFFFFFFF96C298D84539A1F4AD
:10CCB000A033EB2D817D0377F240A463E5E6BCF859
:10CCC00047422CE1F2D1176BF551BF376840B6CB24
:10CCD000CE5E316B5733CE2B169E0F7C4AEBE78E20
:10CCE0009B7F1AFEE242E34F4B60D2273E3CCE3B95
:10CCF000F6B053CCB0061D65BC86987655BDEBB337
:10CD0000E7933AAAD835C65ABF9707006597070038
:10CD1000ED8F0700011101FF01000000000000007D
:10CD2000021702FE6400000068CD0700031704FC30
:10CD30000400000008CE0700000000000000000012
:10CD400000000000010100000100000000000000E0
:10CD500002050000210000000000000000000000AB
:10CD60000000000000000000011104FC04000000AD
:10CD700000000000021104FC04000000000000009C
:10CD8000032104FC0404000000000000041101FF62
:10CD90000100000000000000051102FE0400000078
:10CDA00000000000061104FC040000000000000068
:10CDB000071104FC0400000000000000081701FF38
:10CDC0002200000044CD0700091001FF010000000F
:10CDD000E0CD07000000000000000000000000009F
:10CDE00000000000011704FC7000000014CD0700D3
:10CDF000021704FCB400000020CE07000000000071
:10CE0000000000000000000001010000040000001C
:10CE10000000000000000000000000000000000012
:10CE2000010700007000000014CD0700020100009F
:10CE300001000000000000000305000041000000A8
:10CE400000000000000000000000000000000000E2
:10CE5000982F8A4291443771CFFBC0B5A5DBB5E965
:10CE60005BC25639F111F159A4823F92D55E1CABD9
:10CE700098AA07D8015B8312BE853124C37D0C5567
:10CE8000745DBE72FEB1DE80A706DC9B74F19BC1AF
:10CE9000C1699BE48647BEEFC69DC10FCCA10C249F
:10CEA0006F2CE92DAA84744ADCA9B05CDA88F97683
:10CEB00052513E986DC631A8C82703B0C77F59BFED
:10CEC000F30BE0C64791A7D55163CA066729291419
:10CED000850AB72738211B2EFC6D2C4D130D3853B6
:10CEE00054730A65BB0A6A762EC9C281852C729278
:10CEF000A1E8BFA24B661AA8708B4BC2A3516CC7A6
:10CF000019E892D1240699D685350EF470A06A10DE
:10CF100016C1A419086C371E4C774827B5BCB0342D
:10CF2000B30C1C394AAAD84E4FCA9C5BF36F2E68CB
:10CF3000EE828F746F63A5781478C8840802C78C5A
:10CF4000FAFFBE90EB6C50A4F7A3F9BEF27871C65D
:10CF50004901B952C5EF41DE27476A5527B31CE79F
:10CF60002D1ECB0FA00C3792BE6AB2E99B2403950D
:10CF70006593690B5EF09CFDA5C02CEEF1ECA5A1BC
:10CF8000470A9B3F814C5FD407D8A31404C609D33A
:04CF9000000000009D
:08CF9400ACB4FF7F01000000B6
:10CF9C000000000000000000000000000000000085
:10CFAC000000000000000000000000000000000075
:10CFBC000000000000000000000000000000000065
:10CFCC000000000000000000000000000000000055
:10CFDC000000000000000000000000000000000045
:10CFEC000000000000000000000000000000000035
:10CFFC000090D0030100FFFF258407000184070087
:10D00C000010000000300800419E070000000000E6
:08D01C00D5A80700C9A3070015
:020000020000FC
:020000041000EA
:041014000080070051
:0410180000E00700ED
:0400000370008539CB
:00000001FF
